:1000000047C2000061C200005FC200005DC2000084
:100010005BC2000059C2000057C2000055C2000078
:1000200053C2000051C200004FC200004DC2000088
:100030004BC2000049C20000ADC3000045C2000031
:1000400043C2000041C200003FC200003DC20000A8
:100050003BC2000039C2000037C2000035C20000B8
:1000600033C2000031C20000A0A1A1A01B09A51C41
:10007000A010A0A0201A0111B12C0D0E0216031819
:10008000A00B0A0807060413A00915191412051776
:10009000A0A6A40D0A0F0CA0A01D1BA0A0C0BFBE4F
:1000A00000BDBCBBBAB9B8B7A8A9AAAB0000ADAC3B
:1000B000A0A1A1A01B09A55C7F503B2F205A415154
:1000C000A02C4D4E42564358A04B4A4847464453F5
:1000D000A049555954524557A0A6A40D0A4F4C2E7D
:1000E0007E5D5B2D3A303938403736353433323126
:1000F000A8A9AAAB0000ADACA0A1A1A01B09A57C3A
:100100007F502B3F205A4151B23C4D4E42564358EE
:10011000A04B4A4847464453A04955595452455765
:10012000A0A6A40D0A4F4C3E7E7D7B3D2A30292897
:100130006027262524232221A8A9AAAB0000ADAC64
:10014000A0A1A1A01B09A55C7F703B2F207A617143
:10015000A02C6D6E62766378A06B6A6867666473C4
:10016000A069757974726577A0A6A40D0A6F6C2ECC
:100170007E5D5B2D3A303938403736353433323195
:10018000A8A9AAAB0000ADACA4A1A1A0A01BA51575
:10019000A010A0A0201A0111A02C0D0E0216031809
:1001A000A00B0A0807060413A00915191412051755
:1001B000A0A0A00DA60F0CA0A0A0B1A0A0C0BFBE83
:1001C00008BDBCBBBAB9B8B7A8A9AAAB0000ADAC12
:1001D000A4A1A1A0A01BA515A0503B2F205A4151BE
:1001E000A02C4D4E42564358A04B4A4847464453D4
:1001F000A049555954524557A0A0A00DA64F4C2ECA
:10020000A0A0A02D3A303938083736353433323192
:10021000A8A9AAAB0000ADACA4A1A1A0A01BA515E4
:10022000A0402B3F205A4151A03C4D5E42564358BE
:10023000A04B4A4847464453A04955595452455744
:10024000A0A0A00DA64F4C3EA0A0B23D2A30292868
:100250000827262524232221A8A9AAAB0000ADAC9B
:10026000A4A1A1A0A01BA515A0502B3F205A41512D
:10027000A03C4D4E42564358A04B4A484746445333
:10028000A049555954524557A0A0A00D404F4C3E8F
:10029000A0A0B23D2A302928082726252423222180
:1002A000A8A9AAAB0000ADACA4A1A1A0A01BA51554
:1002B0007F703B2F207A6171A02C6D6E627663781F
:1002C000A06B6A6867666473A069757974726577F4
:1002D000A0A0A00D5E6F6C2EA0A0A02D3A303938E2
:1002E0000837363534333231A8A9AAAB0000ADAC9B
:1002F000A5A20113040607080A0B0C0B0A7FB1A57F
:10030000A4A11A180316020E0D0C0E0FA180A0A0B6
:100310001B010203040506070809000D1E1B1C1D16
:10032000B20911170512141915090F10000D0A8CC6
:10033000A8A9AAAB0000ADACB3978120939A8E8B8D
:100340002D372A382F39A0A0343135323633A0A0CA
:10035000302E2BA0A0A0A0A0A5A241534446474800
:100360004A4B4C3B3A5FA6A5A4A15A584356424E6D
:100370004D3C3E3FA180A0A01B21222324252627FF
:100380002829203D7E5B5C5DB20951574552545986
:1003900055494F50600D0A8CA8A9AAAB0000ADAC1E
:1003A000B3978120939A8E8B2D372A382F39A0A0AE
:1003B000343135323633A0A0302E2BA0A0A0A0A01F
:1003C000A5A24153444647484A4B4C3B3A7FA6A519
:1003D000A4A15A584356424E4D2C2E2FA180A0A0C6
:1003E0001B313233343536373839302D5E5B5C5D46
:1003F000B20951574552545955494F50400D0A8C36
:10040000A8A9AAAB0000ADACB3978120939A8E8BBC
:100410002D372A382F39A0A0343135323633A0A0F9
:10042000302E2BA0A0A0A0A0A5A26173646667686F
:100430006A6B6C3B3A7FA6A5A4A17A786376626E5C
:100440006D2C2E2FA180A0A01B31323334353637CE
:100450003839302D5E5B5C5DB209717765727479F5
:1004600075696F70400D0A8CA8A9AAAB0000ADACED
:10047000B3978120939A8E8B2D372A382F39A0A0DD
:10048000343135323633A0A0302E2BA0A0A0A0A04E
:1004900011241FBECFEFD8E0DEBFCDBF12E0A0E039
:1004A000B1E0EAE5F9E102C005900D92A033B10791
:1004B000D9F723E0A0E3B2E001C01D92A43CB2074B
:1004C000E1F711D70C947D0C9BCD805A813208F056
:1004D00037C0E82FF0E0E158F34F28C7C5C3C6C3C3
:1004E000C9C3CDC3D8C3E0C475C37CC383C38AC3A7
:1004F000A6C1C2C487E063C588E061C589E05FC565
:1005000081E05DC582E05BC583E059C584E057C5E5
:1005100085E055C586E053C584E0C9C285E0C7C201
:1005200086E0C5C287E0C3C288E0C1C289E0BFC21D
:100530008AE0BDC28BE0BBC28CE0B9C28DE0B7C21D
:100540000895815A8D3070F4E82FF0E0E056F34FB3
:10055000EDC6A5C3A6C3C0C439C340C347C34EC379
:1005600071C176C40895682F809133023CC2CF9345
:10057000C82F813A18F0A9DFCF910895F4DF809158
:1005800034028C17C9F3C093340259D4F5CFCF93FA
:10059000C82F8A3041F06C2F8091320224D28C2FE8
:1005A00090E0CF9108958DE0F2DFF5CFCF93809169
:1005B00032024CD2C82F803A41F0809130029091A3
:1005C000310252D18C2FCF910895809133023ED2C7
:1005D000C82FF8CF90E090933102809330020895B5
:1005E000CF93DF93C82FD62F5FD3482F6D2F8C2F3B
:1005F0000DD3DF91CF9108956F927F928F929F924A
:10060000AF92BF92CF92DF92EF92FF920F931F9320
:10061000CF93DF9381E05AD2A82EB92E83E047D240
:1006200000E00F2EFAE07F2EF02D88248394912C89
:100630000F2EF0EA6F2EF02D5AC08C2F90E0F701AC
:10064000E80FF91F20813FEF320F2130D1F03083C6
:10065000D6951695CF5F8BD2C81708F047C0D0FD4E
:10066000ECCF10FFF5CF6C2F802FBADF90913402C2
:100670008913EECF3ED4882359F38091340277DF7B
:10068000E7CFF701E80FF91F708210FF12C0F601E3
:10069000EB54FD4F94010C2E02C0220F331F0A941D
:1006A000E2F78081822B80836C2F802F99DF5FDFC0
:1006B000CFCFF601EB54FD4F94010C2E02C0220F58
:1006C000331F0A94E2F7C9018095908189238083C2
:1006D0006C2F802F85DF813A38F490913402891392
:1006E000B7CF60923402B4CF2CDFB2CF0F5F34D2D9
:1006F0000817C0F4802FF5010995182FC02ED12CB2
:10070000F601EB54FD4FD081D827C0E0C601880F19
:10071000991F880F991F880F991F9C012B5C3D4FD3
:10072000790199CFDF91CF911F910F91FF90EF90B9
:10073000DF90CF90BF90AF909F908F907F906F9001
:10074000089580EA809334020BD16AD33DD280E1D0
:1007500090E019D18093330280E890E014D1809327
:100760003202A5EBB2E0E5E3F2E025EC32E08AE00C
:100770001D928083818382838383848385838683A0
:10078000878338962A173B0799F708953C9A259A4C
:10079000249A08958F9381E08093C6028F911895D3
:1007A0008091C6021092C6020895882311F04498E1
:1007B0000895449A0895882311F02D9A08952D984C
:1007C0000895882311F02C9A08952C980895882371
:1007D00019F0459A3D9A08954598FCCF882319F061
:1007E0003D98459A089545983D9A0895882319F0B3
:1007F000459A3D9A08953D9845980895882319F0A3
:100800002B98239A08952B9AFCCF08950895089564
:10081000882319F02F9A279A08952F98FCCF8823C0
:1008200019F027982F9A08952F98279A08958823CA
:1008300019F02F9A279A089527982F9808952E989F
:10084000269A08952E9A269A08958AE18A95F1F7B4
:1008500000C008952FE788E391E021508040904048
:10086000E1F700C000000895282F392F2115310528
:1008700061F080E090E0EFECF7E03197F1F700C035
:100880000000019628173907B1F70895F8941092DF
:10089000C60287E0809361001092C6028CE787BD94
:1008A00015BC82E084BD80936E0083E085BD80919D
:1008B000C5028BB98FEF8AB91092C502C0DF66DF1F
:1008C00065DF88B1807F88B987B18F6087B92A9842
:1008D000229A299A219A209828987894089598B174
:1008E0008F70907F892B88B929982A9A2A98299AFB
:1008F00020E030E080E0E1E093B19E27492F417095
:1009000050E0BA01022E02C0660F771F0A94E2F788
:10091000862B2A9A2A982F5F3F4F2830310561F79E
:1009200008959091C50289278BB91E9A8AE18A950C
:10093000F1F700C01E9A0895833059F028F48130F1
:1009400039F0823021F4FAC3843009F48EC487C3AD
:10095000B8C327C4982F81E0953008F080E008954F
:100960001092C9021092C8021092C70208958823FB
:1009700044F091E02091C70282170CF090E0892F9B
:10098000089580E00895282F392F8091C702843080
:1009900034F56091C8027091C90240E950E0461BED
:1009A000570B42175307ECF091E0980F9093C70252
:1009B00097E08902F0011124E653FD4F338322832F
:1009C000AB014A515D4F51834083148215821682D8
:1009D000260F371F3093C9022093C80208958FEF66
:1009E00008958FEF0895CF93DF93C82FD62FBFDFE1
:1009F000882349F18C2F0C2E000C990B27E0C202A2
:100A0000F0011124E653FD4F268162817381422F4C
:100A100050E046175707BCF4FC01EE0FFF1FEE0F26
:100A2000FF1FEE0FFF1FE81BF90BE653FD4F8481FC
:100A300090E0A081B181A80FB91FDC93019663D427
:100A400084832F5F2683DF91CF910895CF93C82FA2
:100A50008EDF30EA882339F18C2F0C2E000C990B95
:100A600027E0C202F0011124E653FD4F268130EA4F
:100A70002223C9F0FC01EE0FFF1FEE0FFF1FEE0F48
:100A8000FF1FE81BF90BE653FD4F858190E0A08125
:100A9000B181A80FB91F3C9101966281738133D453
:100AA000858321502683832FCF91089508959FEF4A
:100AB000980F9D3050F4E82FF0E0EE0FFF1FEA583A
:100AC000FC4F0190F081E02D099508959FEF980F5C
:100AD0009D3048F4E82FF0E0EE0FFF1FEA58FC4F7E
:100AE00080819181089586E595E008959FEF980FA4
:100AF0009D3040F4E82FF0E0EE0FFF1FEA58FC4F66
:100B0000608371830895E6E7F3E022E933E086E548
:100B100095E081939193E217F307D9F7E6E7F3E0C5
:100B20008FE694E09383828381E994E095838483C4
:100B30000895643080F4413170F4293060F4E62F78
:100B4000F0E0EE0FFF1FEE0FFF1FED56FC4F80830E
:100B50009183428323830895A7D0E82FF0E0EE0F1E
:100B6000FF1FEE0FFF1FED56FC4F828108959CD0B2
:100B7000E82FF0E0EE0FFF1FEE0FFF1FED56FC4FCA
:100B800083810895CF93DF93D82FE4DE811103C0D2
:100B9000DF91CF910895D093920378DEC0E020E0FA
:100BA00040E06C2F80E090E0C4DFCF5FC430B9F745
:100BB00031D2A9DF8D2FC0DEEBCF90919203981335
:100BC00001C00895DFDFFDCF80E0DCCF809192038C
:100BD0008E7FF3CF809192038160EFCF809192035B
:100BE0008D7FEBCF809192038260E7CF809192035B
:100BF0008B7FE3CF809192038460DFCF809192035B
:100C0000877FDBCF809192038860D7CF982F209188
:100C1000920330E0F901EE0FFF1FEE0FFF1FED56BC
:100C2000FC4F83818823C1F022812223A1F0E42F8D
:100C3000F0E0EE0FFF1FEE0FFF1FED56FC4F70E0D0
:100C4000899F600D711D11240190F081E02DE60F48
:100C5000F71F84910895822F08958093A50361E082
:100C600081FF62E08BE074C181E0F7CF8091A50342
:100C70008260F3CF8091A50392E08927EECF909117
:100C8000A40381E089278093A40361E0913009F4F3
:100C900062E08AE05DC181E08093A303089580E073
:100CA000DCCF1092A3030895E1E08091A5038111A8
:100CB00001C0E0E08091A4038111E2608091A30370
:100CC0008111E460F0E0EE5BFE4F808108951F9398
:100CD000CF93DF93162FC82FD0E0CC0FDD1FCC0FA2
:100CE000DD1FC050DF4FE881F981862F09951A83F7
:100CF000DF91CF911F910895CF93DF93C82FD0E05C
:100D0000CC0FDD1FCC0FDD1FC050DF4FE881F98114
:100D100081E0099581E08A83DF91CF910895CF9397
:100D2000DF93C82FD0E0CC0FDD1FCC0FDD1FC050EC
:100D3000DF4FE881F98180E009951A82DF91CF9138
:100D40000895E82FF0E0EE0FFF1FEE0FFF1FE050B9
:100D5000FF4F61E09281911160E0B9CF282F90910F
:100D600003019923B9F0981779F0E92FF0E0892F62
:100D7000EE0FFF1FEE0FFF1FE050FF4F93819923EF
:100D800059F02913F2CF0895882311F080E00895D7
:100D90008DE008958DE008958DE00895E82FF0E04E
:100DA000EE0FFF1FEE0FFF1FE050FF4F83810895EE
:100DB0001F93CF93DF93C82FD62F142FCFDF9FEF32
:100DC0009C0F9C30C8F48D30E1F0EC2FF0E0EE0F7A
:100DD000FF1FEE0FFF1FE050FF4F9381A82FB0E0E1
:100DE000AA0FBB1FAA0FBB1FA050BF4F13969C9307
:100DF000D383128381E001C080E0DF91CF911F9106
:100E0000089580E0FACFE2E0F1E080E091E09083A5
:100E10008F5F818334968D30D1F71092330108951E
:100E20008DE092E09093A9038093A8039093AB0385
:100E30008093AA039093A7038093A60308958091BB
:100E4000AA039091AB039093A7038093A603089500
:100E50001092A9031092A8038091AA039091AB036A
:100E60008234910541F01092AB031092AA031092C4
:100E7000A7031092A60308958DE092E09093A90332
:100E80008093A8038091AA039091AB0382349105CB
:100E900051F08DE092E09093AB038093AA0390937E
:100EA000A7038093A60308958091A6039091A703BA
:100EB0008334910530F48091AA039091AB03892B80
:100EC00051F482E490E09093AB038093AA03909353
:100ED000A7038093A60308958091A8039091A90386
:100EE0009093AB038093AA039093A7038093A603E8
:100EF00008958091A6039091A703009799F09C0113
:100F000021503109019731F03093A7032093A603B4
:100F100080E0089582E490E09093A7038093A60375
:100F200081E0089580E008950F931F93CF93082FD9
:100F3000192FC62F662341F08C2FF80109958C2FAD
:100F40002DDFC82F8111F8CFCF911F910F910895F8
:100F5000CF93E82FF0E0EE0FFF1FE455FC4FC08168
:100F60006330F1F048F0643081F06530B9F46C2FF3
:100F700081EA96E0D9DF12C06130E1F0623071F4AD
:100F80006C2F8FE896E0D0DF09C06C2F81EA96E0E5
:100F9000CBDF60DC6C2F81EA96E0C6DFCF9108954D
:100FA0006C2F81EA96E0C0DF50DC6C2F81EA96E07E
:100FB000BBDFF4CF6C2F8CE796E0B6DFEFCFE82FE6
:100FC000F0E0EE0FFF1FE455FC4F6181C1CF0F939E
:100FD0001F93CF93DF93162F042F9FEF980F9B3013
:100FE00028F0DF91CF911F910F910895C82FD0E085
:100FF000FE01EE0FFF1FE455FC4F422F6081812F51
:10100000D7DE882371F3CC0FDD1FC455DC4F188366
:101010000983E7CFF8DEECEAF3E084EC93E0118299
:1010200010823296E817F907D1F70895CF93DF932E
:10103000CDB7DEB7AE014B5F5F4FFA0161917191A1
:10104000AF0184E391E08CD1DF91CF9108958AE4E0
:1010500091E09F938F93EADF0F900F90089588E2BD
:10106000B9DA60E080E057D062E081E054D061E01E
:1010700082E051D063E083E04ED067E278E08DE01B
:1010800035DD6BEF78E08CE031DD21E040E06AE0B7
:1010900087E09DDF20E040E06CE08AE098DF21E01F
:1010A00043E068E081E093DF20E044E063E082E039
:1010B0008ECF8AE491E09F938F93B8DF0F900F90CB
:1010C000089588E287DA60E081E025D062E081E07F
:1010D00022D061E082E01FD063E083E01CD069E5AC
:1010E00078E08DE003DD6BEF78E08CE0FFDC21E061
:1010F00040E06AE087E06BDF20E040E06CE087E002
:1011000066DF21E043E068E081E061DF20E044E069
:1011100063E082E05CCFE82FF0E0EE0FFF1FE35AC0
:10112000FE4F28E049E08081918103CD85E691E082
:101130009F938F937BDF0F900F90089588E24ADA98
:1011400060E080E07FD062E081E07CD061E082E01E
:1011500079D063E084E076D06BEF78E08CE0C6DC99
:1011600066E978E08DE0C2DC20E040E06AE08AE0F9
:101170002EDF20E040E06CE088E029DF21E043E062
:1011800068E081E024DF20E044E063E082E01FDFEC
:1011900076CD82E891E09F938F9348DF0F900F9078
:1011A000089588E217DA60E081E04CD062E081E0E7
:1011B00049D061E083E046D063E084E043D06BEF48
:1011C00078E08CE093DC69EC78E08DE08FDC20E067
:1011D00040E06AE087E0FBDE20E040E06CE088E091
:1011E000F6DE21E043E068E081E0F1DE20E044E06B
:1011F00063E082E0ECCE89E991E09F938F9316DF64
:1012000084EA91E09F938F9311DF84EB91E09F93A9
:101210008F930CDF8EED91E09F938F9307DF84EF28
:1012200091E09F938F9302DF8AE092E09F938F93E8
:10123000FDDE8DB79EB70C960FB6F8949EBF0FBE1D
:101240008DBF0895E82FF0E0EE0FFF1FEA5EFD4F1F
:1012500028E049E0808191816CCC80E292E09F930C
:101260008F93E4DE0F900F90089528E04DE060E04A
:1012700088E294E05EDC28E04DE062E080EC93E000
:1012800058DC28E04DE061E088E593E052DC28E09E
:101290004DE063E080EF92E04CDC88E29BD920E0F7
:1012A00040E06AE08AE093DE20E040E06CE08BE022
:1012B0008EDE21E045E061E083E089DE20E045E06C
:1012C0006BE083E084DE21E043E068E081E07FDEE4
:1012D00021E044E064E082E07ADED1DCB3DA6DE262
:1012E00079E08DE003CC2DDA01C086D959DA882364
:1012F000E9F35CD9C82F803AC1F382E0E7DBFC0157
:101300008C2F0995F2CF97FB072E16F4009406D088
:1013100077FD08D011D007FC05D03EF4909581955B
:101320009F4F0895709561957F4F0895EE0FFF1FB1
:101330000590F491E02D0994AA1BBB1B51E107C055
:10134000AA1FBB1FA617B70710F0A61BB70B881F55
:10135000991F5A95A9F780959095BC01CD010895E4
:10136000AFE0B0E0E5EBF9E094C26C017B018A01EB
:10137000DC0117961C921E92169713968C9181FF92
:10138000DEC12AE0522EF6019381F70193FD85918B
:1013900093FF81917F01882309F471C0853239F46C
:1013A00093FD859193FF81917F01853221F4B601F0
:1013B00090E0DED1E8CF912C612C712CFFE1F71584
:1013C00008F445C08B32C1F1F0F48032B9F18332B8
:1013D00009F43AC0833609F487C0833709F490C012
:1013E000833509F0B0C0F801A190B1908F01692D4B
:1013F00070E076FC02C06FEF7FEFC501A3D14C0116
:10140000689477F85EC08D32E1F0803351F020EDC2
:10141000280F2A3048F18E3209F038C0689476F8E7
:1014200002C0689470F8F70193FD859193FF819154
:101430007F018111C3CF32C0689471F8689472F84B
:10144000F2CF689473F8EFCF689474F8ECCF77FC20
:1014500025C020ED280F2A3070F476FE05C0959C3B
:10146000200D1124922EDFCF659C200D1124622EB9
:10147000689475F8D8CF8E3249F476FECFCFD60176
:1014800016968D919C912F96EFE01FC28C3619F421
:10149000689477F8C8CF883609F4C5CF982F9F7D18
:1014A0009554933008F096CF0C5F1F4F8FE38983DC
:1014B00088248394912CAE014F5F5F4F5A01E894CA
:1014C00077F873FC05C0862D90E08816990630F1F8
:1014D0008114910449F5662009F455CFB60180E2E4
:1014E00090E046D16A94F7CFD8018C9189830E5F42
:1014F0001F4F88248394912CFE0131965F01DFCF2A
:10150000D801AD90BD908D01692D70E076FC02C0D0
:101510006FEF7FEFC50121D14C01D1CFB60180E241
:1015200090E026D16A94CFCFF50177FC859177FEC4
:1015300081915F01B60190E01BD161106A94F1E0E6
:101540008F1A9108C5CF843619F0893609F07DC00D
:10155000F80177FE73C061917191819191918F0132
:10156000272D2F76822E97FF09C090958095709534
:1015700061957F4F8F4F9F4F689487F82AE030E046
:10158000AE014F5F5F4F5A0123D18A19A82EBA2CA2
:10159000782C86FE0CC0E89470F8A91440F484FE00
:1015A00005C082FC03C0782D7E7E772EB92C74FE98
:1015B000A1C0FE01EA0DF11D8081803309F093C0C6
:1015C000872D897E782E73FC0EC070FEA1C09A2CE8
:1015D000B61418F4960C9B18B62C862D8B196B1428
:1015E00008F480E0B80EB61408F094C06B1874FECE
:1015F00093C0B60180E390E0BBD072FE08C088E5DE
:1016000090E071FC02C088E790E0B601B1D0A91467
:1016100008F48FC0AA94B12C9FEFA91AB90ADE0171
:1016200011964D01AA0EBB1EF50182915F01B60114
:1016300090E09ED08A149B04B9F74DCF61917191CF
:10164000072E000C880B990B8ACF872CE89484F81E
:101650002AE030E0853769F0572D597F852E803795
:1016600069F110F5883569F18F3609F008CF28E067
:1016700030E0F80187FE2DC081919191A191B19147
:101680008C879D87AE87BF878F01BE016F5F7F4FBD
:101690005B01AB016C857D858E859F8599D08A190C
:1016A000A82EE89487F873CF883709F0E8CE84FE37
:1016B00002C0689482F820E130E0DBCF689484F8BF
:1016C000F6CF74FE03C0652F6660862E20E132E0FF
:1016D000D0CF81919191AC0160E070E04C875D8743
:1016E0006E877F87D1CF72FC02C0B3946CCFB39466
:1016F000B39469CF872D8678882309F464CFF5CF1A
:10170000B60180E290E034D083948614C8F365CFAC
:101710008B2CFBCF612C6BCF872D8678882309F427
:1017200076CF8BE271FE80E277FC8DE2B60190E02D
:101730006DCFB60180E390E01BD09A9468CF8FEF15
:101740009FEFA1CEFC010590615070400110D8F7C9
:10175000809590958E0F9F1F0895FC0161507040F9
:1017600001900110D8F7809590958E0F9F1F0895D6
:101770000F931F93CF93DF93182F092FEB018B81CA
:1017800081FD09C01FEF0FEF812F902FDF91CF91C7
:101790001F910F91089582FF14C02E813F818C818B
:1017A0009D81281739073CF4E881F981CF01019622
:1017B0009983888310838E819F8101969F838E8376
:1017C000E3CFE885F985812F0995892BA1F3DACF3D
:1017D000FA01AA27283051F1203181F1E8946F9362
:1017E0006E7F6E5F7F4F8F4F9F4FAF4FB1E03ED008
:1017F000B4E03CD0670F781F891F9A1FA11D680FA6
:10180000791F8A1F911DA11D6A0F711D811D911DD8
:10181000A11D20D009F468943F912AE0269F11244D
:101820003019305D3193DEF6CF010895462F4770B1
:10183000405D4193B3E00FD0C9F7F6CF462F4F700C
:10184000405D4A3318F0495D31FD4052419302D06A
:10185000A9F7EACFB4E0A695979587957795679510
:10186000BA95C9F700976105710508959B01AC0110
:101870000A2E06945795479537952795BA95C9F737
:10188000620F731F841F951FA01D08952F923F9212
:101890004F925F926F927F928F929F92AF92BF9280
:1018A000CF92DF92EF92FF920F931F93CF93DF932C
:1018B000CDB7DEB7CA1BDB0B0FB6F894DEBF0FBE89
:1018C000CDBF09942A88398848885F846E847D84D6
:1018D0008C849B84AA84B984C884DF80EE80FD80D8
:1018E0000C811B81AA81B981CE0FD11D0FB6F8944E
:1018F000DEBF0FBECDBFED010895F894FFCF8C027F
:101900006E026F0270027102720273028C02740224
:10191000750276027702790278027A027C027E02F0
:10192000800282028402860288028A028C028E026F
:10193000900292029402960298029A029C029E02DF
:10194000A902B202B202B202AA02AB02B202AC0215
:0A195000AD02AE02AF02B102B00218
:10195A0005040000E7030000EE030000F6030000A0
:10196A00FE0300000604000007040000080400004B
:10197A000F04000017040000D5030000DB03000079
:10198A00E10300000000000200000000C70200009E
:10199A00000000010201030303035B4B65796D61DB
:1019AA00703A20636C61737369635D0A004001B029
:1019BA0000F80068005B4B65796D61703A204170F0
:1019CA00706C6520322028752F6C2063617365293D
:1019DA005D005B4B65796D61703A204170706C6592
:1019EA00203220434150535D003130204745542076
:1019FA0041240D0032302041203D204153432841EB
:101A0A0024290D0033302049462041203C2033321E
:101A1A00205448454E2041243D2243544C2B222B2E
:101A2A00434852242841202B203634290D003430D3
:101A3A00203F2227223B41243B2227203D20223BD4
:101A4A00413A0D0035302049462041203C3E2033A2
:101A5A0020474F544F2031300D00363020454E4438
:101A6A000D52554E0D00A802D001600218028801DD
:101A7A005B4B657962643A20536F6C2D32305D009E
:00000001FF
